:020000020000FC
:0200000011C02D
:02000E0058C0D8
:0A001400009186008CC0219618951B
:10002000119618950FEE0AB90FEE0BB90FE307B949
:1000300000E008B900E304B90EE105B90FEF0DBF08
:1000400004E00EBFFF2480E091E0CC27DD27AA2743
:10005000BB272FEF0FE6102F1801280138014801A8
:1000600058016801E02E71E000E004BD00E005BD2C
:1000700000E006BD01E000936E0000E00093800008
:1000800001E40093810001E200936F0002E000931D
:10009000B00006E00093B1000FE60093B30002E069
:1000A0000093700000E800BF07E80093640001E0DF
:1000B00003BF01E005BB01E206BB78948895FECF43
:1000C000F8B802E105B9E0E3F4E0E70FFF1D099499
:1000D0007A95C1F477E08A95B1F0A3F480E02FEF30
:1000E0000FE6102F18012801380148015801680156
:1000F000E02EF5BC91E0AA27BB27F6BC01E005BBCA
:1001000000E206BB189501E200936F0000E206BB17
:10011000189507E005BDCC27DD27F0928500F09209
:10012000840084E6992701E000936F0001E006BB9C
:10013000189510918700903061F70000F5BC2E01F2
:10014000180136B5AD0105B30170400F5F1D01E127
:10015000200E3F1C4F1C5F1C20920D0130920E019F
:1001600040920F01509210010DD091E084E6AA2731
:10017000BB27F6BC01E200936F0001E005BB01E282
:1001800006BB1895002711271801280138014801DE
:1001900058016801E02EFF24199902C0ACD201C0B9
:1001A00081D100E0201600EA300602E740060EE4A6
:1001B000500608E1600609E070068F049F04AF0452
:1001C000BF04CF04DF04EF0480F00AE0E02ED02E5D
:1001D000C02EB02EA02E902E802E702E602E502E6F
:1001E000402E302E202E2FEF47C100270093000114
:1001F00000930101009302010093030100930401A5
:100200000093050100930601009307010093080184
:100210000093090100930A0100930B0100930C0164
:1002200000E0201600E1300605EA400604ED500625
:1002300008EE60067F0488F000E0201A00E1300A32
:1002400005EA400A04ED500A08EE600A7F080091B2
:100250000C01039500930C01E3CF00E0201608EE9B
:10026000300606E7400608E4500607E1600680F025
:1002700000E0201A08EE300A06E7400A08E4500AB7
:1002800007E1600A00910B01039500930B01E5CF94
:1002900000E0201604EE30060BE0400604E55006B0
:1002A00002E0600680F000E0201A04EE300A0BE065
:1002B000400A04E5500A02E0600A00910A01039531
:1002C00000930A01E5CF00E020160AEC30060AE9A7
:1002D00040060BE350066F0478F000E0201A0AECA9
:1002E000300A0AE9400A0BE3500A6F08009109013D
:1002F000039500930901E7CF00E0201601EE3006D8
:1003000005EF400605E0500670F000E0201A01EE0F
:10031000300A05EF400A05E0500A009108010395F4
:1003200000930801E9CF00E8201606E9300608E945
:10033000400600E0500670F000E8201A06E9300A96
:1003400008E9400A00E0500A009107010395009374
:100350000701E9CF00E4201602E430060FE0400672
:1003600060F000E4201A02E4300A0FE0400A009135
:100370000601039500930601EDCF00EA201606E87A
:10038000300601E0400660F000EA201A06E8300A74
:1003900001E0400A00910501039500930501EDCFAE
:1003A00000E1201607E2300600E0400660F000E1C0
:1003B000201A07E2300A00E0400A00910401039588
:1003C00000930401EDCF08EE201603E0300650F054
:1003D00008EE201A03E0300A009103010395009310
:1003E0000301F1CF04E6201600E0300650F004E6E9
:1003F000201A00E0300A00910201039500930201E7
:10040000F1CF0AE0201640F00AE0201A0091010125
:10041000039500930101F5CF309001014090020156
:1004200050900301609004017090050180900601D6
:1004300090900701A0900801B0900901C0900A01B6
:10044000D0900B01E0900C01222700279016A00607
:10045000B006C006D006E00679F0232C342C452CDB
:10046000562C672C782C892C9A2CAB2CBC2CCD2CA0
:10047000DE2CEE242395E9CF022D24D2202E032D4D
:1004800021D2302E042D1ED2402E052D1BD2502EEF
:10049000062D18D2602E072D15D2702E082D12D2DF
:1004A000802E089500E0309F100100E3509F40012E
:1004B00005EE509F300100E0509F200102E1509F67
:1004C000900CA11C0CE9509F700C811C9F1CAF1C50
:1004D00000E4509F500C611C7F1C8F1C9F1CAF1CA4
:1004E00002E1409F800C911CAF1C00E3409F700C08
:1004F000811C9F1CAF1C0CE9409F600C711C8F1C61
:100500009F1CAF1C05EE409F500C611C7F1C8F1C74
:100510009F1CAF1C00E4409F400C511C6F1C7F1CB3
:100520008F1C9F1CAF1C00E0409F300C411C5F1CC7
:100530006F1C7F1C8F1C9F1CAF1C02E1309F700C36
:10054000811C9F1CAF1C00E3309F600C711C8F1C32
:100550009F1CAF1C0CE9309F500C611C7F1C8F1C32
:100560009F1CAF1C05EE309F400C511C6F1C7F1C64
:100570008F1C9F1CAF1C00E4309F300C411C5F1C83
:100580006F1C7F1C8F1C9F1CAF1C30910D01409174
:100590000E0150910F016091100119E48894002719
:1005A00000930001009301010093020100930301F5
:1005B00000930401009305010093060100930701D5
:1005C00000930801221C331C441C551C661C771C1C
:1005D000881C991CAA1C1A9509F48CC00091000172
:1005E000001F0093000100910101001F0093010111
:1005F00000910201001F0093020100910301001FFE
:100600000093030100910401001F00930401009175
:100610000501001F0093050100910601001F0093D2
:10062000060100910701001F0093070100910801D6
:10063000001F0093080100910001031B00930001BB
:1006400000910101040B0093010100910201050BCF
:100650000093020100910301060B00930301009136
:1006600004010F0900930401009105010F09009393
:100670000501009106010F09009306010091070191
:100680000F0900930701009108010F090093080169
:1006900078F500910001030F009300010091010122
:1006A000041F0093010100910201051F0093020144
:1006B00000910301061F00930301009104010F1D27
:1006C00000930401009105010F1D009305010091A5
:1006D00006010F1D00930601009107010F1D0093F5
:1006E0000701009108010F1D0093080188946ACF4B
:1006F000089468CF08958A0140910E0150910F012E
:1007000000930E0110930F01032F30910D016091A2
:10071000100100930D0100E5309F100100E5509F8E
:10072000200103EC609F300100E5409F300C411C2C
:100730005F1C6F1C7F1C00E5609F500C611C7F1CC0
:1007400003EC309F300C411C5F1C6F1C7F1C03ECC2
:10075000409F400C511C6F1C7F1C03EC509F500CA1
:10076000611C7F1C30910D0140910E0150910F01D1
:1007700011E3889400270093000100930101009386
:100780000201009303010093040100930501221C60
:10079000331C441C551C661C771C1A9509F45FC059
:1007A00000910001001F0093000100910101001F52
:1007B0000093010100910201001F009302010091CA
:1007C0000301001F0093030100910401001F009327
:1007D000040100910501001F009305010091000133
:1007E000031B0093000100910101040B0093010120
:1007F00000910201050B00930201009103010F0912
:1008000000930301009104010F090093040100917A
:1008100005010F090093050100F500910001030F88
:100820000093000100910101041F00930101009158
:100830000201051F00930201009103010F1D0093A7
:100840000301009104010F1D0093040100910501B3
:100850000F1D0093050188949ACF089498CF0895AE
:1008600007C006C00BC010C015C01AC01FC024C0EE
:10087000263009F42C982BB82D9A2ACC253009F46F
:100880002C983BB8409A24CC243009F42C984BB8CF
:10089000419A1ECC233009F42C985BB8429A18CCAC
:1008A000223009F42C986BB8439A12CC213009F409
:1008B0002C987BB8449A0CCC203009F42C988BB837
:1008C000459A06CC0C3008F00BE0F8E0E6EDE00FBE
:1008D000FF1D0491089580E94460292202E8002068
:0208E000E70629
:00000001FF
